:100200004F726967696E616C2046696C653A20704F
:10021000726F6A6563742E6865780D0A4F75747025
:10022000757420446174653A20323030392F30358E
:100230002F32370D0A4F75747075742046696C65DE
:100240003A20657039343331783428646267292E56
:100250006865780000000000000000000000000059
:10026000000000000000000000000000000000008E
:100270000000000000000000000000000000002D51
:102499000D0A205B48444D492076312E3362204D88
:1024A90061747269785D0D0A0D0A000D0A004861B0
:1024B90072647761726520494F20696E6974696138
:1024C9006C20646F6E652E2E2E2E2E2E2E2E2E0D26
:1024D9000A0053595354454D3A204F5554505554B9
:1024E90020312069732073656C65637465640D0A16
:1024F9000053595354454D3A204F55545055542083
:10250900322069732073656C65637465640D0A0014
:1025190053595354454D3A204F555450555420332F
:102529002069732073656C65637465640D0A0053D3
:10253900595354454D3A204F555450555420342041
:1025490069732073656C65637465640D0A0053597A
:102559005354454D3A2052554E204B4559206973E5
:102569002073656C65637465640D0A00535953548F
:10257900454D3A20506F72742053776974636869C6
:102589006E672064657465637465642E2E2E0D0A6A
:102599000053595354454D3A204F555450555420E2
:1025A90025642073776974636820746F20494E50DD
:1025B9005554202558206973207365740D0A0052FB
:1025C9005332333220434D443A20537472696E6753
:1025D90020427566666572204F766572666C6F7704
:1025E9000D0A002573202558202558202558202517
:1025F90058005357430073776300525332333220E4
:10260900434D443A2053776974636820746F2049B5
:102619004E5055542025580D0A004552524F523AF2
:1026290020506172616D32206F766572666C6F77CA
:102639000D0A004552524F523A20506172616D3174
:10264900206F766572666C6F770D0A0053454C00F2
:1026590073656C00525332333220434D443A205350
:10266900656C65637420746865204F5554505554E2
:102679002025640D0A00505752007077720052539A
:1026890032333220434D443A2053656C65637420DC
:1026990074686520706F77657220737461747573DF
:1026A9002069732025640D0A005253540072737413
:1026B90000525332333220434D443A2053797374D4
:0B26C900656D2052657365740D0A00FA
:0E3D390041F82B0042F81F000042F82600005F
:10327C0090F82CE0FEA3E0FFC39404EE64809480ED
:10328C002290F828E0FF2421F582E434F8F583221B
:10329C0090F82CE0FEA3E02421F58274F83EF5832F
:1032AC0022780D7CF87D017BFF120755EF2290F8F8
:1032BC002CE0FCA3E0FF2421F58274F83CF583E0BC
:1032CC0022740AF074002FF58274F83EF583E4F052
:1032DC0074302FF58274F83EF58374FFF090F82D5E
:1032EC00E004F022780D7CF87D017BFF120755EF8E
:1032FC0022E4F0A3F090F82CF0A3F02290F82CE04C
:10330C0004F022780D7CF87D017BFF120755EF222B
:10331C00A3F0A37401F0A32274302FF58274F83E4D
:10332C00F5832290F82574FFF0E490F828F0C21190
:10333C00C210C20F2278007CF87D017B017AF879EB
:10334C00217E007F0422C390F82DE0940490F82C89
:10335C00E0648094802290F8047402F022780D7C52
:10336C00F87D017BFF120755EF227BFF7A26793C13
:01337C00222E
:100A1200E4FF1244387D017F407E0212381E7BFFC4
:100A22007A2479991240147BFF7A2479B412401403
:100A32007BFF7A4379AAE4FF1244EB7B007C007DC2
:100A420064122A6A7BFF7A0079561244DFE4FF12AD
:100A520041B11226D47A2479B712113290F80412D5
:100A6200330012327C501074212F1232A51232CD73
:100A720070F012330880EB12332FC390F827E09402
:100A82000A90F826E09400405B1232FD12327C504C
:100A920038124388EF90F82C6017E0FEA3E0FF24A1
:100AA20030123327E025E04401FD123324EDF080BB
:100AB2000EE0FEA3E02430123327E0FF25E0F0121F
:100AC20032E970C812330880C3120003EF90F82590
:100AD2006009E0FF25E04401F08005E0FF25E0F039
:100AE200D20F8002C20F90F804E014600D14605718
:100AF20024026003020E51020C3A301021C2107F10
:100B0200011242CBEF24DB70151210BE12327C5060
:100B12000A12106570F612330880F1123362300F38
:100B22002090F825E064FE70181210BE12327C503C
:100B32000A12106570F612330880F1123362020E47
:100B420051438701020E51E412330112327C4003F9
:100B5200020C3074212F1232A5E024F5602E1460AD
:100B62004914607324036003020C1E1210B5600363
:100B7200020BC61210C96003020BFD1210D26002F2
:100B8200802D12110190F82C604B80531210C96015
:100B920003020BFD1210D2600280141211016005D3
:100BA20090F82C803A1210B5804212110A60069019
:100BB200F82C020C10121120600590F82C802012E3
:100BC2001129600280267D087F01123959EF90F8C1
:100BD2002C60028029803F121120600B90F82C12A9
:100BE200329F740DF08035121129600590F82C8027
:100BF200257D087F01123959EF600B90F82C1232D3
:100C02009F740BF0801612110A90F82C60081232B1
:100C12009F740CF0800612329F740AF01232BAFDF1
:100C220012315D1232E97003123308020B4D300F9C
:100C32006690F825E0B4FE06121139020E26E4127F
:100C4200330112327C5050123324E0647F703D90A5
:100C5200F82C1232A1E024F5601514601A14601FFA
:100C62002403702174212F1232A5740BF080161206
:100C7200329C740CF0800E12329C740DF0800612BD
:100C8200329C740AF01232BAFD12315D1232E970EE
:100C920003123308020C44201003020D9FC2107F7E
:100CA200011242CBEF1205700D7F050D0E060D6A83
:100CB200070D77080D900C0D02150CEA170CE71BB7
:100CC2000CE11C0CFB1D0CF4200CDE230CD8240CB4
:100CD200ED2700000D9F121139020D7A020D6A12E2
:100CE2001113020D7A020D7F020D9012328D740AD9
:100CF200801312328D740B800C12328D740C8005AD
:100D020012328D740DF090F828E080527BFF7A2524
:100D1200795712401412328DE0FEB40A0B74212F5F
:100D2200123294740BF08031EEB40B0C90F828E080
:100D3200123292740CF0802112328DE0FEB40C0B50
:100D420074212F123294740DF0800EEEB40D0A90BD
:100D5200F828E0123292740AF090F828E0FF12327A
:100D620092E0FD12315D80357A2479DB12113290E6
:100D7200F828F080281211137401F080207BFF7A8A
:100D820025791912401490F8287402F0800F7BFF25
:100D92007A25793812401490F8287403F0123341FE
:100DA2001208F8EF601C123341120350E490F82944
:100DB200F0D21190F81FF0A3F07BFF7A257975121B
:100DC200401490F829E0146060046003020E51C3DD
:100DD20090F820E094E890F81FE0940340711232FA
:100DE200FD7BFF7A25799A90F82CE0FCA3E0FD24A4
:100DF20001FEE43C90F837F0A3CEF074212D1232BC
:100E0200C4FF90F839E4F0A3EFF01240141232BAA2
:100E1200FD12337D1232E97003123308123352404D
:100E2200C090F8297401F08026C390F820E094B8AD
:100E320090F81FE0940B40171232FD1232BAFD12E5
:100E4200337D1232E9700312330812335240EC122E
:100E5200114090F82AEFF0F47003020A7CE0FFA33D
:100E6200E0FE04F0740D2EF582E434F8F583EFF021
:100E720090F82BE0D39412400E7BFF7A2579C812AA
:100E82004014E490F82BF090F82AE0FF640A60081E
:100E9200EF640D6003020A7CE490F82BF090F86591
:100EA20074FFF0A37425F074EC12331C74FFF07419
:100EB2008012331C74F8F0A3740512331D74F8F019
:100EC200A3740712331D74F8F0A3740912331D744E
:100ED200F8F0A3740BF07B017AF8790D12198EE405
:100EE20090F810F07A2579FB1232AD60097A2579F3
:100EF200FF1232AD70657A26790390F8071210DB83
:100F0200EE94004050D3EF9403EE94005047A3E0D8
:100F1200FEA3E0FFC3940AEE94004030D3EF940D99
:100F2200EE9400502790F805A3E0FFFD90F828F01A
:100F320090F807A3E0FC74212D123294ECF0742196
:100F42002F123294E0FD12315D020A7C7BFF7A2679
:100F520079230210031233760210037A267955128E
:100F620032F060097A2679591232F0702E7A267997
:100F72005D90F8051210DBEE94004019D3EF940354
:100F8200EE9400501090F805A3E0123292E0FD12A8
:100F9200337D020A7C1233760210037A26797F129D
:100FA200330F60097A26798312330F705A7BFF7AE6
:100FB20026798790F805E0FFA3E090F837CFF0A3F9
:100FC200EFF012401490F805E0FAA3E0FB4A700C2F
:100FD2001238BF90F8047401F0020A7CEB64014AF3
:100FE200701C124221E412330112327C500A121098
:100FF2008D70F612330880F1123362020A7C1233CA
:1010020076124014020A7C7A2679B2123369600C95
:101012007A2679B61233696003020A7C7BFF7A264C
:1010220079BA1240141226D4E412330112327C50DF
:101032001074212F1232A51232CD70F012330880B3
:10104200EB12332F1238BF124221E4123301123253
:101052007C500A12108D70F612330880F11233623E
:10106200020A7C74002FF58274F83EF583E4F09056
:10107200F82CE0FCA3E02421F58274F83CF583E02F
:10108200FD12315D90F82DE004F02274002FF582FC
:1010920074F83EF583E4F090F82CE0FCA3E0242100
:1010A200F58274F83CF583E0FD12315D90F82DE095
:1010B20004F0227D047F01123959EF22124221E409
:1010C20090F82CF0A3F0227D087F01123959EF220B
:1010D2007D017F01123959EF227BFFE0FFA3E090EF
:1010E200F837CFF0A3EFF012401490F806E024FF97
:1010F200F090F805E034FFF0E0FEA3E0FFC3227DAC
:10110200027F01123959EF227D017F01123959EF15
:10111200227BFF7A2479FA12401490F828227D0269
:101122007F01123959EF227D047F01123959EF22D2
:0E1132007BFF124014E4221238BF90F8042212
:10005600AE07E4FF1242CBBFEB09EE7006EDB4101B
:0400660002D2102290
:1043AA0090F827E004F0700690F826E004F0301147
:1043BA000E90F820E004F0700690F81FE004F02256
:103003004552524F523A2043616E6E6F7420666987
:103013006E64204F555450555425640A0D0053597E
:103023005354454D3A204F55545055542025642050
:10303300416464723D307825302E325820666F75B6
:103043006E640A0D004552524F523A204F75747008
:10305300757420506F7274204572726F722C204FFA
:1030630075747075742025642025580D0A00455227
:10307300524F523A2055706461746520545245474B
:10308300204572726F722C20535725642077726922
:10309300746520307839300D0A004552524F523A48
:1030A30020494943206661696C65642C207374610F
:1030B3007475733D50656E64696E67200D0A004533
:1030C30052524F523A20494943206661696C656404
:1030D3002C207374617475733D4E6F416374200DBE
:1030E3000A004552524F523A2049494320666169CA
:1030F3006C65642C207374617475733D54696D65DC
:10310300204F7574200D0A004552524F523A204900
:103113004943206661696C65642C2073746174751E
:10312300733D4172626974726174696F6E4C6F733F
:1031330073200D0A004552524F523A204949432009
:103143006661696C65642C207374617475733D30BA
:0A3153007825302E3258200D0A00B6
:103F7900F07B017AF9790E90F904E4F0A37402F068
:103F8900E4A3F07D7AFF2290F911E0FEA3E0240179
:103F9900FFE43E90F837F0A3EF227BFF90F950E061
:103FA9002401FEE43390F837F0A3CEF022E490F92F
:0E3FB9000EF0A32290F90E7401F0A374902272
:1026D400E4FB7D01FF1241EB7D021228A37D011270
:1026E40028A37B017D017F04121F047B017D027FEF
:1026F40004121F047D207F0212287D7D407F021278
:102704001F047B027D807F02121F047D0412285F58
:102714007D087F05121F047B027D017F05121F04C3
:102724007D0212285F7D407F05121F047D807F0596
:1027340012287D7D107F05121F047B027D207F05FA
:10274400121F047D041228697D08E4FF121F047D12
:10275400011228697D02E4FF121F047D40122891B2
:102764007D80E4FF121F047D101228917D20E4FF78
:10277400121F047B027D027F06121F047B027D046C
:102784007F06121F047F0212289B7D041228737D8A
:10279400087F02121F047D101228737D087F061221
:1027A4001F047D041228AB7D081228ABE4FB7D01D5
:1027B4007F01121F047F0112289B7F011244D31250
:1027C4003FBDF0E490F911F0A3F090F911E0FEA3FD
:1027D400E0FFC39404EE9400400302285EEE703AD6
:1027E400EF14601214601E1460232403702C12284A
:1027F40085122D3C8006122885122BD57D807F0200
:10280400122BD580151228B3122D3C80061228B342
:10281400122BD57D807F02122D3C7F011244BB1206
:102824003F7A1228BF90F90DEFF07BFF60097A30F0
:102834007903123F90800E7A307921123F90F0A3F1
:10284400E4F0A3747AF012401490F912E004F070EA
:102854000690F911E004F00227CE227B027F0512D4
:102864001F047B02227B02E4FF121F047B0222E48A
:10287400FB7F02121F04E4FB227B02121F047B0273
:10288400227D207F02122D3C7D407F02227B02E4C8
:10289400FF121F047B0222E4FB7D02121F04227B31
:1028A400017F08121F0422E4FB7F01121F04227D12
:0B28B400207F02122D3C7D407F02229D
:104221007D047F06122D3C7D027F06122BD57D0277
:104231007F08122BD57D017F08122BD57D017F04CC
:0F424100122BD57D027F04122BD57F0A0244BBBE
:1038BF007D047F06122BD57D027F06122D3C7D02E3
:1038CF007F08122D3C7D017F08122D3C7D017F0466
:1038DF00122D3C7D027F04122D3C7D047F05122B9F
:1038EF00D57D087F05122BD57D017F05122BD57D48
:1038FF00027F05122BD57D407F05122BD57D807F52
:10390F0005122BD57D107F05122BD57D207F05123B
:10391F002BD57D04E4FF122BD57D08E4FF122BD5A8
:10392F007D01E4FF122BD57D02E4FF122BD57D40E4
:10393F00E4FF122BD57D80E4FF122BD57D10E4FF21
:0A394F00122BD57D20E4FF022BD5DA
:10337D0090F951EDF090F950EFF014601214601EB9
:10338D001460232403702C123434122D3C80061249
:10339D003434122BD57D807F02122BD5801512343B
:1033AD0040122D3C8006123440122BD57D807F02B9
:1033BD00122D3C7F011244AF90F951E024F56011BC
:1033CD0014601C14601224037025123FB674FC8027
:1033DD0013123FB674FD800C123FB674FE800512B9
:1033ED003FB674FF123F791228BF90F90DEFF090A0
:1033FD00F90DE060177A307948123FA390F951E04A
:10340D00FF90F839E4F0A3EFF012344C123FBD12E7
:10341D003F791228BF90F90DEFF0600A7A3079717B
:10342D00123FA312344C227D207F02122D3C7D4091
:10343D007F02227D207F02122D3C7D407F022212D1
:0B344D00401490F90DE0FF12406122D6
:10315D00AC05EF14604C1470030231EB14700302D4
:10316D00322E240360030232727D047F05122BD5AB
:10317D007D087F05122BD57D017F05122BD57D0294
:10318D001232736011146012146013240360030271
:10319D0032727D0480437D08803F7D01803B7D023E
:1031AD0080377D407F05122BD57D807F05122BD575
:1031BD007D107F05122BD57D2012327360111460A6
:1031CD0012146013240360030232727D40800A7D65
:1031DD008080067D1080027D207F0502326F7D0488
:1031ED00E4FF122BD57D08E4FF122BD57D01E4FF02
:1031FD00122BD57D02E4FF122BD5EC24F5601014B3
:10320D0060131460162403705C7D04E4FF80537D0D
:10321D0008E4FF804D7D01E4FF80477D02E4FF80DF
:10322D00417D40E4FF122BD57D80E4FF122BD57D2F
:10323D0010E4FF122BD57D20E4FF122BD5EC24F5E5
:10324D006010146013146016240370197D40E4FFA0
:10325D0080107D80E4FF800A7D10E4FF80047D20D6
:0F326D00E4FF122D3C227F05122BD5EC24F52215
:10438800EF14600E14600F146010240370137D0284
:10439800800A7D0480067D0880027D107F02123924
:0243A800592298
:080003007D087F061239592225
:1040610090F958EFF024FE601214601714601C24BC
:104071000370207BFF7A30799D802B7BFF7A30792A
:10408100C280237BFF7A3079E5801B7BFF7A31790F
:104091000B80137BFF7A31793890F958E0FF90F863
:0A40A10037E4F0A3EFF01240142200
:103D4700182B000000000000000000000000000029
:0A3D57000000000000000000000062
:103ED60085128385138222860308E6FA08E64A4B92
:103EE6002208E6FA08E6F9020596A3E0FEA3E0FF3B
:103EF6002290FFFF12059CEFF0C2A922AA06AB078B
:103F060090F959E025E0227C001203C5EF22F8A6BD
:103F16000308A60208A60122F8E6FE08E6FFE4FC6E
:023F2600FD227A
:102A6A0090FFFF12059CEBF090FFFE12059CECF024
:102A7A00A3EDF0123EF7E58954FCFE123ED6E0FBC8
:102A8A004EF5899000031205C0E044C0F58B90F919
:102A9A005DE014605A147003022B412402600302A1
:102AAA002B93123ED6123EF0EE54FE7009758C1628
:102ABA00EEC313EF805F123ED6123EF0EE54FC7066
:102ACA0010758C2DEF7802CEC313CE13D8F9022BD2
:102ADA0082123ED6123EF0D394EAEE9415500B754C
:102AEA008CFC7D16123F0D022B82AF03022B8C1237
:102AFA003ED6A3E0FEEE700C758C0E123ED6A3A352
:102B0A00E0022B82EE54FE700F758C1D123ED6A386
:102B1A00E0C313A3E0138060123ED6123EF0D394B2
:102B2A00EFEE9410500A758CFE7D11123F0D80480D
:102B3A00123ED6E0FF804B123ED6A3E0FEEE700BAB
:102B4A00758C10123ED6A3A3E0802DEE54FE700FB2
:102B5A00758C21123ED6A3E0C313A3E01380191289
:102B6A003ED6123EF0D394EFEE94105010758CFEC0
:102B7A007C007D0F1203C5EF14F58D800C123ED632
:102B8A00E0FF1243CA7F00803CAF8C123ED6E0FDC4
:102B9A0025E02423F8760008A607AF8DED25E0246A
:102BAA0043F8760008A6077401A805088002C33313
:102BBA00D8FCF5887410A805088002C333D8FC42F3
:0B2BCA0089D2A97F0190000402059C45
:1043CA00123EF7123ED6E0FF7410A807088002C317
:0E43DA0033D8FCF45289D2A990000102059C50
:0B44EB00EF75F003A4242B123F1422F5
:0B44F600EF75F003A42437123F1422DE
:1035310090F959EFF0FBC2A9E58954FC4BF589AF2D
:103541008C784F760008A607AF8DE4FCFDFE784B22
:10355100120564EB25E02443123F1E784B120557F8
:10356100C3EF9BFFEE9AFEED99FDEC98FCC004A918
:1035710005123F022423123F1ED00012041AC00478
:10358100C005123F022424F9C3E7785096FF19E7DA
:103591001896FEE4FCFDD001D000EB2FFFEA3EFEC1
:1035A100ED39FDEC38FC784B12056490F95DE014BF
:1035B100601C14602424027033E47F19FEFDFC7842
:1035C1004B12055712041AE47B207A018014784BC0
:1035D10012054BE47B0FFA8009784B12054BE47B13
:1035E10011FAF9F81204A5784B120564D2A9784DA5
:0635F100E6FE08E6FF22E1
:03000B0002345864
:10345800C0E0C0F0C083C082C0D075D000C000C03A
:1034680001C002C003C004C005C006C007308812EE
:10347800782B123EDD6005782B123EE77588010235
:103488003516308912782E123EDD6005782E123EF0
:10349800E7758802023516308A127831123EDD60EF
:1034A800057831123EE7758804023516308B11789D
:1034B80034123EDD60057834123EE7758808804E88
:1034C800308C117837123EDD60057837123EE7758B
:1034D8008810803A308D11783A123EDD6005783ACE
:1034E800123EE77588208026308E11783D123EDD29
:1034F8006005783D123EE77588408012308F0F785E
:1035080040123EDD60057840123EE7758880D0079E
:10351800D006D005D004D003D002D001D000D0D03E
:09352800D082D083D0F0D0E03253
:08450B00E5FF54077851F62288
:05004E0012450B002229
:1043E80012450BE6FF700476098008EFB4010C78DB
:0C43F8005176027851E660031680F8222E
:1043650012450BE6FF7004760C800FEFB40106785A
:104375005176048005EFB40209227851E6600316F0
:0343850080F8229B
:1043190012450BE6FF700476178012EFB401067898
:104329005176098008EFB4020C785176027851E68B
:0643390060031680F8226B
:103FC70090F95DE014601314602624027036E5FF53
:103FD700540770387851760D802AE5FF540714602E
:103FE7000904702878517615801A78517603801461
:103FF700E5FF54071460090470127851761A80049B
:0D400700785176057851E660031680F822A6
:103CBB0090F95DE014602714604424027067E5FFFF
:103CCB00540714600D14601024027061785176450E
:103CDB0080537851761B804D785176058047E5FFF0
:103CEB00540714600D146010240270417851765FF4
:103CFB00803378517628802D7851760C8027E5FF1C
:103D0B0054071460101460131460162403701E788B
:103D1B0051766D80107851762F800A7851760F800E
:0E3D2B0004E47851F67851E660031680F82221
:1039F200301304D2AED2BE90F95DE0146030146090
:103A02005624027079E5FF540714601014601314F1
:103A12006016240370707851767E80627851763712
:103A2200805C785176138056785176018050E5FF9C
:103A3200540714601014601314601624037047783E
:103A42005176A980397851764C80337851761E8030
:103A52002D785176078027E5FF5407146010146013
:103A6200131460162403701E785176C080107851AA
:103A72007658800A7851762480047851760A7851F3
:073A8200E660031680F82244
:102EA300301304D2AED2BE90F95DE0146078147092
:102EB30003022F9324026003022FF2E5FF5407B4A9
:102EC30007004003023002902ED1F8282873022E07
:102ED300E6022EED022EF7022F01022F0B022F1511
:102EE300022F1F78527603022F85785276010876D7
:102EF30084022FF2785276000876BC022FF27852C1
:102F03007600087658022FF2785276000876260269
:102F13002FF27852760008760D022FF2785276005F
:102F2300087601022FF2E5FF5407B40700400302BD
:102F33003002902F3CF8282873022F51022F5B0296
:102F43002F65022F6F022F78022F81022F8A78526A
:102F53007604087607022FF2785276010876FD028E
:102F63002FF2785276000876F9022FF27852760023
:102F7300087676807A7852760008763580717852B2
:102F83007600087615806878527600087604805FAC
:102F9300E5FF5407B407005066902FA3F828287361
:102FA300022FB8022FC1022FCA022FD0022FD9023B
:102FB3002FE2022FEB78527604087689803178521B
:102FC300760208763E80287852760180167852760B
:102FD3000008768780197852760008763D8010784D
:102FE30052760008761980077852760008760678BC
:102FF30053E61846600908E6161870F31680F022A7
:10448F007851760A7851E6166005122EA380F52230
:10449F00785176647851E6166005122EA380F522C6
:0C44AF00AE071FEE60051239F280F52206
:0C44BB00AE071FEE6005122EA380F52254
:0C44C700AE071FEE600512448F80F52246
:0C44D300AE071FEE600512449F80F5222A
:103D610046F91400000000000006140000000000E5
:013D71000051
:103A890075BC01C390F90AE094A890F909E0946122
:103A99002214FF781AE67814FD08E6FA08E6F5829A
:103AA9008A8302059A7814860308E6FA08E64A4BDF
:103AB9002290F904E0FEA3E0FF90F907E0FCA3E0FF
:103AC900FDC39FEC9E22F5B7E490F909F0A3F0221B
:103AD900E5BC540690F90BF022ED5401C43333547C
:103AE900C022781C0806E618860622241AF582E404
:103AF90034F9F5832290F909E004F02290F90B7466
:103B090003F022E490F907F0A3F02290F901E0FB19
:073B1900A3E0FAA3E0F9228A
:1041EB00EF6019D2BAED6006D2B6D2B78004D2B462
:1041FB00D2B543BB04E490F91BF08017D2B9ED6044
:10420B0006D2B2D2B38004D2B0D2B143BB02E49097
:06421B00F91AF002425006
:10425000EF600543BB01800353BBFEEDB4020CEBE2
:104260005403C454F0FF123AE2800C123AE2448044
:0B427000FFEB5403C454F04FF5B722DD
:1041390090F947EBF0EF6014D2BAED6006D2B6D22F
:10414900B78004D2B4D2B543BB048012D2B9ED60B2
:1041590006D2B2D2B38004D2B0D2B143BB021200AC
:0C4169002690F947E0F5B3A3E0F5B6227C
:10002600E5BB54FE4FF5BBEDB40208123AE3442A91
:10003600F5B122123AE244AAF5B175B4FF75B21FC2
:0400460043B101229F
:10445000EF75F003A42414F582E434F9F583EBF04E
:07446000A3EAF0A3E9F0223A
:1001EF00EF75F003A42414F8A60308A60208A601CD
:0101FF0022DD
:1028BF0090F8FFEFF0A3EDF0A3EBF0A3EAF0A3E99C
:1028CF00F0123B0CA3F0A3F0A3F090F8FFE0FE1280
:1028DF003AF4E060037F0122741A2E123AF6740163
:1028EF00F0E5BB54FE4EF5BB75BC0190F906E02038
:1028FF00E12E90F900E0F5BDE5B754F14402123A2C
:10290F00CFE5BC20E00D122A567003123AFE123AA0
:10291F008C40EE123A895005123AD98003123B05CA
:10292F0090F90BE06003022A4790F900E020E003E2
:10293F000229C5123B0C123ABA4003022A1890F929
:10294F000BE06003022A18EF24FFFFEE34FFFEEDC9
:10295F00B50715ECB5061190F906E020E00AE5B7CA
:10296F0054F1440AF5B78008E5B754F14406F5B7BA
:10297F00123AD1E5BC20E00D122A567003123AFE2E
:10298F00123A8C40EE123B1490F907E0FEA3E0F5EB
:10299F00828E83E5BF1203A3123A895005123AD9EA
:1029AF008003123B0590F908E004F0700690F907D8
:1029BF00E004F0022945123B0C123ABA504B90F941
:1029CF000BE07045123B148D828C83120376F5BE9B
:1029DF00E5B754F14406123ACFE5BC20E00D122AB8
:1029EF00607003123AFE123A8C40EE123A8950058B
:1029FF00123AD98003123B0590F908E004F07006F3
:102A0F0090F907E004F00229C890F906E020E028C9
:102A1F00E5B754F1440E123ACFE5BC20E00D122A6F
:102A2F00607003123AFE123A8C40EE123A8950054A
:102A3F00123AD98003123B0590F8FFE0123AF4E402
:102A4F00F090F90BE0FF2212004E90F90AE004F02B
:0B2A5F002212004E90F90AE004F02261
:03004B00023BACC9
:103BAC00C0E0C0F0C083C082C0D075D000C000C0DF
:103BBC0001C002C003C004C005C006C00790F95A7A
:103BCC00E5BBF053BBFEE5B230E113123AAE60092F
:103BDC00123AEB700106123A9A75B202802BE5B2DA
:103BEC0030E310781C7600087600781AA6B575B20A
:103BFC00088016E5B230E011123AAE6009123AEBC9
:103C0C00700106123A9A75B20190F95AE0F5BBD0E0
:103C1C0007D006D005D004D003D002D001D000D0FC
:0A3C2C00D0D082D083D0F0D0E03277
:03005300023778F9
:10377800C0E0C0F0C083C082C0D075D000C000C017
:1037880001C002C003C004C005C006C00790F95BB1
:10379800E5BBF0E5BB54FE4401F5BBE5B230E11EE4
:1037A8007817123AB06012781E123AED70010614BA
:1037B800FF781BE67817123AA175B2028037E5B296
:1037C80030E310781E7600087600781BA6B575B22F
:1037D800088022E5B230E01D7817123AB0601378FD
:1037E8001E123AED70010614FF781BE6FD781712D9
:1037F8003AA275B20190F95BE0F5BBD007D006D0CC
:1038080005D004D003D002D001D000D0D0D082D0CF
:0638180083D0F0D0E03285
:10427B00EBF0A3EAF0A3E9F02290F940E0FBA3E016
:10428B00FAA3E0F92275A102439A03439C03539BC3
:09429B00FC227B017AFF798022EC
:10381E0090F931EEF0A3EFF0A3EDF090F95DE01426
:10382E00600F146014240270507F007ED07D0280E1
:10383E000E7F807EA97D0380067FB07E1E7D047C78
:10384E0000E5FF5407F9F8120537E47B20FAF9F882
:10385E001240F5C006C00790F931E0FEA3E0FBAAC6
:10386E0006E4F9F8D007D0061240F5C3E49F90F9AC
:10387E0035F074049E90F934F0438780759850901B
:10388E00F934E0F5BAA3E0F5AA75A101E5A1B401FA
:10389E000512429080037595037E007F127D007B9A
:1038AE00017AF879ED12091C90F933E06002D2AC7E
:0138BE0022E7
:103F280090F93612427BA3ECF0A3EDF0E4FFFE75A6
:103F3800A101E5A1B401051242908003759503D350
:103F480090F93AE09FEE6480F890F939E06480983F
:103F5800401E90F9361242878F828E83120376F5BF
:103F680099E59830E1FB5398FD0FBF00010E80CF13
:013F78002226
:1044200090F95CEFF07B017AF9795C7D017C0012F8
:084430003F2890F95CE0FF2237
:1041750090F93B12427BE4A3F0A3F090F93B124285
:1041850087A3E0FEA3E0F5828E83120376FF60131A
:1041950012442090F93FE004F070E090F93EE0040D
:0C41A500F080D890F93EE0FEA3E0FF227D
:1040140090F83412427B90F85F7401F0A374F8F0C6
:10402400A37437F090F834E0F9A3E0FAA3E090F930
:104034002BC912427C90F85FE0F9A3E0FAA3E09068
:10404400F92EC912427C12429D1240AB12429D12BB
:0D405400000EAC06AD0712429D123F28225F
:03002300023E8218
:103E8200C0E0C083C082C0D075D000C004C005C0ED
:103E920007E59830E02F90F8FDE0FF2401FDE433C0
:103EA200FCA3E06D7001EC601974ED2FF582E4342F
:103EB200F8F583E599F090F8FDE004F0E0B4100223
:103EC200E4F05398FED007D005D004D0D0D082D0F1
:043ED20083D0E03287
:1042A4007FFF90F8FEE0FE90F8FDE06E601874ED7C
:1042B4002EF582E434F8F583E0FF90F8FEE004F094
:0742C400E0B41002E4F02257
:103E2C0090F94012427BA3ECF0A3EDF0E4FDFCD33F
:103E3C0090F944E09DEC6480F890F943E06480983C
:103E4C00402F1242A4EFF460F91242848D828C83CD
:103E5C00EF1203A3EFB40A12ED1D70011C12428481
:103E6C008D828C83E41203A380070DBD00010C80AE
:063E7C00BEAE04AF0522FA
:103D72004DF8DE000000FF000000000000F0E0004F
:103D820041F8DA0041F8DB0041F8EB0041F8EC00C1
:083D920041F8DD0041F8D90001
:103C3600C454F0FEEF4EFFF090F94DE024DEF5821D
:103C4600E434F8F58322E0FF90F94EE022E0FE909E
:103C5600F957E022E090F953FEE033333354F8226B
:103C660075A101E5A1640122E090F94EFEE0C4547D
:103C7600F0FD22E0FD90F957E0FCED6C22E0FF2418
:103C8600FB24FB22C454F0FD90F8D9E05DFDEE2242
:103C960090F957E0FFEE6F2290F94EE0540FF0A333
:103CA600E0FF22E0FEC454F05FFFEE4FF022F4FE88
:053CB600EF5EF0EE22BC
:101F040090F94EEDF0A3EBF090F94DEFF014604929
:101F1400146079147003021FB6147003021FD524D1
:101F2400FA700302200814700302204F240B60038C
:101F34000220B690F94FE0FF700790F94EE042FCA2
:101F440022EF90F94EB40205E042C88004E0F45256
:101F5400C890F94EE0F452FC2290F94FE0FF70076C
:101F640090F94EE042FD22EF90F8DAB40212123CEE
:101F74004CFEEF4EFF90F8DA123C3DE05F42FD224A
:101F8400123C4C90F8DA123CB452FD2290F94FE026
:101F9400FF700790F94EE042FE22EF90F94EB40232
:101FA40005E042D88004E0F452D890F94EE0F452AF
:101FB400FE2290F94FE07012123C3EC083C08212A0
:101FC4003C4CFEEF4ED082D083F0123C3EE0F5B0A4
:101FD4002290F94FE0FF700790F94EE042F322EFB0
:101FE40090F8DBB40212123C4CFEEF4EFF90F8DB8B
:101FF400123C3DE05F42F322123C4C90F8DB123C71
:10200400B452F322123C9E7013123C3EC083C08231
:10201400123C6EEE4DD082D083F08028EF90F8EB26
:10202400B4020E123C4C90F8EB123C36123CA980E0
:1020340013123C4CC454F0F4FEEF5E90F8EB123CE7
:102044003DE05EF0123C3EE0F58A2290F94EE05409
:102054001CF0A3E0FF7018123C3EC083C082E090E5
:10206400F94E123C5EFDEE4DD082D083F0803CEF01
:1020740090F8ECB40220123C4C33333354F8FEEFA6
:102084004EFF90F8EC123C3DE0FE33333354F85FDE
:10209400FFEE4FF08015123C4C33333354F8F4FE0A
:1020A400EF5E90F8EC123C3DE05EF0123C3EE0F551
:1020B400C122123C66706E90F94D123C8350072485
:1020C400FE602C0221DF12433F90F94FE0FF7007BE
:1020D40090F94EE0429B22EF90F94EB40205E042A3
:1020E4009C8004E0F4529C90F94EE0F4529B2290C0
:1020F400F94FE0FF700790F94EE0429722EF90F815
:10210400DDB40212123C4CFEEF4EFF90F8DD123C9F
:102114003DE05F429722123C4CF4FEEF5E90F8DD06
:10212400F0EE52972290F94DE0FF24FA60331460E8
:1021340042146061240360030221DF90F94FE0FE42
:10214400700790F94EE0429B22EE90F94EB40205DE
:10215400E0429C8004E0F4529C90F94EE0F4529BDF
:102164002290F94FE090F94E7004E0429422E0F49A
:1021740052942290F94FE0701574DE2F123C44C043
:1021840083C082123C4CFEEF4ED082D083F0123CCE
:102194003EE0F59522123C9E7013123C3EC083C073
:1021A40082123C6EEE4DD082D083F08028EF90F8FE
:1021B400D9B4020E123C4C90F8D9123C36123CA908
:1021C4008013123C4CC454F0F4FEEF5E90F8D91224
:0C21D4003C3DE05EF0123C3EE0F5AD2228
:10433F00EF24FA6011146012146013146014240433
:10434F007013E4F5A12275A1012275A1022275A1B6
:06435F00032275A10422F7
:10395900AB05AA07EA14601914601B14601D1460F2
:103969001F24FA6020146022240B7023E5805BFF7A
:1039790022E5905BFF22E5A05BFF22E5B05BFF2219
:10398900E5F25BFF22E58A5BFF22E5C15BFF2212BC
:103999003C667032EA24FB24FB500624FE600C804E
:1039A90047AF0212433FE59A5BFF22E58F5470FA55
:1039B900758F7090F8DCE591F0E4F58FE04591F0B2
:1039C9008A8FE05BFF22EA24FA600F146011146009
:1039D9001324037013E59A5BFF22E5935BFF22E54D
:0939E900955BFF22E5AD5BFF22B6
:102BD50090F952EFF0A3EDF090F952E0FF123C426C
:102BE500E04DF0EF14602114603414603B14604232
:102BF50024FA605414607B240B6003022C9E90F928
:102C050052123C41E0F5802290F953E0FF90F8DA4A
:102C1500E05F42FD90F952123C41E0F5902290F9B7
:102C250052123C41E0F5A02290F952123C41E0F5E8
:102C3500B02290F953E0FF90F8DBE05F42F390F9A2
:102C450052123C41E0F5F22290F952E0FF123C426B
:102C5500C083C082E090F953123C7290F8EBE05DBE
:102C6500FDEE4DD082D083F074DE2F123C44E0F5AA
:102C75008A2290F952E0FF123C42C083C082123C86
:102C85005AFD90F8ECE05DFDEE4DD082D083F074F6
:102C9500DE2F123C44E0F5C122123C66704390F9E8
:102CA50052123C83500724FE6010022D3B12433F15
:102CB50090F952123C41E0F59A2290F952E0FF1248
:102CC5003C42C083C082123C5AFD90F8DDE05DFDB8
:102CD500EE4DD082D083F074DE2F123C44E0F591A6
:102CE5002290F952E0FF24FA601414601B1460224C
:102CF5002403704274DE2F123C44E0F59A2290F9C9
:102D050052123C41E0F5932290F952123C41E0F514
:102D1500952290F952E0FF123C42C083C082E0FE4A
:102D250090F953E0123C8A4DD082D083F074DE2FA7
:072D3500123C44E0F5AD2261
:102D3C0090F954EFF0A3EDF090F954E0FF123C42FF
:102D4C00E0FEEDF4FDEE5DF0EF146021146035143F
:102D5C00603C14604324FA6056146077240B6003C3
:102D6C00022E0290F954123C41E0F5802290F95465
:102D7C00123C41E0F59090F955E0FF90F8DAE05FF5
:102D8C00F452FD2290F954123C41E0F5A02290F946
:102D9C0054123C41E0F5B02290F954123C41E0F55C
:102DAC00F290F955E0FF90F8DBE05FF452F32290DB
:102DBC00F954E0FF123C42E0FEF58A74DE2F123C1F
:102DCC0044C083C08290F955E0C454F0FF90F8EBF6
:102DDC00022E9790F954E0FF123C42E0FEF5C174CC
:102DEC00DE2F123C44C083C08290F955123C5FFF29
:102DFC0090F8EC022E97123C66703E90F954123CFF
:102E0C0083500724FE6010022EA212433F90F95407
:102E1C00123C41E0F59A2290F954E0FF123C42E05A
:102E2C00FEF59174DE2F123C44C083C08290F9559C
:102E3C00123C5FFF90F8DD805290F954E0FF24FAC9
:102E4C00601414601B1460222403704A74DE2F1269
:102E5C003C44E0F59A2290F954123C41E0F593225F
:102E6C0090F954123C41E0F5952290F954E0FF1290
:102E7C003C42E0FEF5AD74DE2F123C44C083C082B0
:102E8C0090F955E0C454F0FF90F8D9E05FF4FFEEF0
:072E9C005FD082D083F02219
:1021E00090F957EDF090F956EFF0146044146076D2
:1021F0001470030222871470030222A824FA7003C9
:102200000222DD147003022330240B6003022382B8
:1022100090F956E0FF123C42C083C082123C53FD4D
:10222000EE6DD082D083F074DE2F123C44E0F58056
:102230002290F956E0FF123C42123C53FDF4FCEEB2
:102240005CF59090F8DAE05D62FD74DE2F123C449C
:10225000C083C082123C96D082D083F090F956128F
:102260003C41E0F5902290F956E0FF123C42C083D9
:10227000C082123C53FDEE6DD082D083F074DE2F0D
:10228000123C44E0F5A02290F956E0FF123C42C017
:1022900083C082123C53FDEE6DD082D083F074DE99
:1022A0002F123C44E0F5B02290F956E0FF123C4278
:1022B000123C53FDF4FCEE5CF5F290F8DBE05D625D
:1022C000F374DE2F123C44C083C082123C96D0824D
:1022D000D083F090F956123C41E0F5F22290F95685
:1022E000E0FF123C42123C53F4FDEE5DF58A74DED1
:1022F0002F123C44C083C08290F957E0C454F0FFD1
:1023000090F8EBE05FFFEE6FD082D083F090F9564B
:10231000E0FF123C42C083C082123C53540FFDEEDA
:102320006DD082D083F074DE2F123C44E0F58A2217
:1023300090F956E0FF123C42123C53F4FDEE5DF57D
:10234000C174DE2F123C44C083C08290F957123C06
:102350005FFF90F8ECE05FFFEE6FD082D083F090EB
:10236000F956E0FF123C42C083C082123C53541C19
:10237000FDEE6DD082D083F074DE2F123C44E0F588
:10238000C122123C66706890F956123C83500724B3
:10239000FE602702249812433F90F956E0FF123C5A
:1023A00042C083C082123C53FDEE6DD082D083F0D8
:1023B00074DE2F123C44E0F59A2290F956E0FF12A9
:1023C0003C42123C53FDF4FCEE5CF59190F8DDE0EC
:1023D0005D629774DE2F123C44C083C082123C962B
:1023E000D082D083F090F956123C41E0F5912290D2
:1023F000F956E0FF24FA602B146046146061240350
:10240000600302249890F956E0FE123C42C083C05B
:1024100082123C79D082D083F074DE2E123C44E0EC
:10242000F59A2290F956E0FE123C42C083C0821217
:102430003C79D082D083F074DE2E123C44E0F593D8
:102440002290F956E0FE123C42C083C082123C79D1
:10245000D082D083F074DE2E123C44E0F5952274D5
:10246000DE2F123C44C083C082123C53123C8A6D62
:10247000D082D083F074DE2F123C44C083C082E04F
:10248000FF90F957E0540FFEEF6ED082D083F090AA
:09249000F956123C41E0F5AD22C1
:0C3D9A00C11241F9490043F94A00000041
:1044040090F94AE0FBA3E0FAA3E0F9EA494B2290D1
:0C441400F94AA3E0FAA3E0F5828A8322B3
:1041B10075A101E5A1B4011BEF24FE600C14600E92
:1041C1002403702375A49C801E75A4DC801975A43A
:1041D100FC801443F580EF24FE6009240270087509
:0A41E100A4B8800375A4F8D2BD2233
:0C44DF0090F94AEBF0A3EAF0A3E9F02208
:1042CB0030120CEF70037F862290F949E0FF2275C4
:1042DB00A101E5A1B40107EF04F5A6AFA722EF708A
:0742EB0003AFA622AFA722DA
:03006B00023DB59E
:103DB500C0E0C0F0C083C082C0D075D000C000C0D4
:103DC50001C002C003C004C005C006C007C2127509
:103DD500A101E5A164017019F5A6124404602AE564
:103DE500A530E6047F0180027F00124413ADA78051
:103DF500151244046013E5A530E6047F0180027FB7
:103E0500001244137D1012059A43A580D007D006F1
:103E1500D005D004D003D002D001D000D0D0D082BC
:073E2500D083D0F0D0E032A1
:063DA60041F95D01C113AB
:0645230090F95DEFF022AB
:10443800EF6005D213758680E5FFB430037F012253
:0844480075FF30D2AF7F0022A6
:08451300301304D2AED2BE2227
:101C2700444247434D4420537472696E672042759E
:101C3700666665722046756C6C0D0A002573202553
:101C470058202558202558202558006275730044D0
:101C57004247434D44206275733A204275733D30C5
:101C67007825302E32582C20506F72743D307825ED
:101C7700302E32582C2053706565643D30782530FE
:101C87002E32580D0A0063697200444247434D449F
:101C9700206369723A20436F64653D307825302EA2
:101CA70032580D0A0077723100444247434D4420B1
:101CB7007772313A2049443D307825302E32582CFE
:101CC700205265673D307825302E32582C204461EC
:101CD70074613D307825302E32580D0A0072643118
:101CE70000444247434D44207264313A2049443D01
:101CF700307825302E32582C205265673D307825B4
:101D0700302E32582C2053697A653D307825302E95
:101D170032582C20446174613D200028526561646B
:101D2700206E756D626572206578636565642061F4
:101D3700206D6178206F6620256420627974657351
:101D470029000D0A002000307825302E32582C202B
:101D57000074623100444247434D44207462313A73
:101D67002049443D307825302E32582C2052656763
:101D77003D307825302E32582C204D61736B3D3025
:101D87007825302E32582C20446174613D0030781C
:101D970025302E32580D0A00636231004442474312
:101DA7004D44206362313A2049443D307825302E36
:101DB70032582C205265673D307825302E32582C0A
:101DC700204D61736B3D307825302E32582C2044DE
:101DD7006174613D0077723200444247434D4420AD
:101DE7007772323A2049443D307825302E32582CCC
:101DF700205265673D307825302E34582C204461B9
:101E070074613D307825302E32580D0A00726432E5
:101E170000444247434D44207264323A2049443DCE
:101E2700307825302E32582C205265673D30782582
:101E3700302E34582C2053697A653D307825302E62
:101E470032582C20446174613D0074623200444270
:101E570047434D44207462323A2049443D30782547
:101E6700302E32582C205265673D307825302E347D
:101E7700582C204D61736B3D307825302E32582C0D
:101E870020446174613D0063623200444247434D20
:101E970044206362323A2049443D307825302E325F
:101EA700582C205265673D307825302E34582C2029
:101EB7004D61736B3D307825302E32582C204461AC
:101EC70074613D004552524F523A204949432066BA
:101ED70061696C65642025642C2049494341646429
:101EE700723D307825302E32582C20526567416478
:0D1EF70064723D307825302E32580D0A00FF
:083DAC0041F8D40041F8D200F7
:10006E00A3F090F8B9E0FF90F8BCE0FCA3E090F9A3
:10007E0022FD7B017AF879C0E4F0A304F02278C067
:10008E007CF87D017BFF120755EF227BFF7A1D79ED
:10009E004E90F8D6E024C0F582E434F8F583E0FF04
:1000AE00E490F837F0A3EFF02290F924E090F926CF
:1000BE00FDE0FBA3E0FAA3E0F9A3E0FFA3E090F9D3
:1000CE0004CFF0A3EFF02278C07CF87D017BFF1205
:1000DE000755EF2278C07CF87D017BFF120755EFA4
:1000EE002290F8C0F090F8B9E0FF90F8BBE07AF8F3
:1000FE0079C090F929FD7B01E4F0A32278C07CF849
:10010E007D017BFF120755EF2290F8BBE0FEA3E0C6
:10011E004EF0A3E0F022F0A3EDF0A3EBF0A3EAF093
:10012E00A3E9F090F8D5E4F0A3740AF0E4A3F0A3E9
:10013E00F022A3F0A37401F0A322E0FEA3E0FF904F
:10014E00F8D5E0FCA3E0FDC39FEC9E22E0FFE49017
:10015E00F839F0A3EFF022E0FFA3E0CF90F83BF0E8
:10016E00A3EFF022E0FD7B017AF879C0A3E0FFA3B4
:10017E00E022D390F8D6E0940090F8D5E0940022D7
:10018E00C390F8D8E0940390F8D7E094002278C09A
:10019E007CF87D017BFF120755EF22A3E024FDF0D2
:1001AE0090F8D5E034FFF02290F8B9E0FF90F8BB5C
:1001BE00E0227BFF90F8B8E0FFA3E0227BFF7A1DE0
:1001CE0079492290F8C0E0FF90F8BDE02290F8C087
:1001DE00E0FF90F8BFE0227BFF7A1D799590F8C082
:0101EE0022EE
:101140001242A490F95EEFF0F4700302146FE0FF16
:1011500090F8D4E0FE04F074C02EF582E434F8F583
:1011600083EFF090F8D4E0D39412400E7BFF7A1C0A
:101170007927124014E490F8D4F090F95EE0FF640F
:101180000A6008EF640D600302146FE490F8D4F075
:1011900090F86574FFF0A3741CF07443120140745E
:1011A000FFF0748012014074F8F0A374B81201418A
:1011B00074F8F0A374BA12014174F8F0A374BC126D
:1011C000014174F8F0A374BEF07B017AF879C01283
:1011D000198EE490F8C3F07A1C795212008C701EBC
:1011E0007A1C79561214751201B6FD90F8BDE0FB19
:1011F0001241EB90F8B9E090F8D2F002146F7A1C2B
:10120000798D12008C703F7A1C79911201C0CF1237
:1012100000AF124014D21290F8B9E090F949F09062
:10122000F94AE0FBA3E0FAA3E0F9EA494B700302B4
:10123000146F90F94AA3A3E0F5828A837D10E4FF3E
:1012400012059A02146F7A1C79AC1200D5701E7ABE
:101250001C79B012147590F8BDE090F8C0F012013E
:10126000B690F92912007F1236BB02146F7A1C79EE
:10127000E41200D560030213077A1C79E81201C05A
:1012800090F837CFF0A3EFF090F8BAE0FFA3E0CFEB
:1012900012015D90F8BC120165124014D390F8BDA4
:1012A000E0941290F8BCE09400400312157890F896
:1012B000B9E04401FFC00790F8BB12017290F92910
:1012C000CFF0A3EFF0D0071236BBEF600302146F2C
:1012D00090F8D5F0A3F090F8BC1201485026ED54D8
:1012E0000F70061201CA12401490F8D6E05407702D
:1012F0000312158C12009912159670DA90F8D5E049
:1013000004F080D20214067A1D79581200E2702788
:101310007A1D795C12152B1236BBEF600302146F35
:101320001201D1FEEF6E1200EF04F01236BBEF6037
:101330000302146F0214347A1D799F1200E27028A0
:101340007A1D79A312152B1236BBEF600302146FBE
:101350001201D1F4FEEF5E1200EF04F01236BBEF83
:10136000600302146F0214347A1D79DC12010A70D2
:10137000171201177A1D79E01214A890F8BFE01235
:10138000006E1235F702146F7A1E791412010A707A
:101390007B1201177A1E79181214A8D390F8BFE0B7
:1013A000941290F8BEE09400400312157890F8B9BA
:1013B000E04401FFC00790F8BCE0FCA3120172906A
:1013C000F922CFF0A3EFF0D0071235F7EF60030258
:1013D000146F90F8D5F0A3F090F8BE120148502693
:1013E000ED540F70061201CA12401490F8D6E05462
:1013F00007700312158C12009912159670DA90F886
:10140000D5E004F080D21201CA02146C7A1E795120
:1014100012019C70281201177A1E79551214DB12E2
:1014200035F7EF704A1201DBFEEF6E12006E1235D7
:10143000F7EF703B1201E51200AC02146C7A1E79D2
:101440008E12019C70291201177A1E79921214DBF8
:101450001235F7EF70191201DBF4FEEF5E12006E29
:101460001235F7EF70091201E51200AC124014902A
:10147000F95EE0FF227BFF90F8B8E0FFA3E090F870
:1014800037CFF0A3EFF090F8BAE0FFA3E090F8397F
:10149000CFF0A3EFF090F8BCE0FFA3E090F83BCFD3
:1014A000F0A3EFF0124014227BFF90F8B8E0FFA306
:1014B000E090F837CFF0A3EFF090F8BCE0FFA3E0A6
:1014C00090F839CFF0A3EFF090F8BEE0FFA3E090E2
:1014D000F83BCFF0A3EFF0124014227BFF90F8B856
:1014E000E0FFA3E090F837CFF0A3EFF090F8BCE076
:1014F000FFA3E090F839CFF0A3EFF090F8BEE0FF43
:10150000A3E090F83BCFF0A3EFF012401490F8B9AD
:10151000E04401FF90F8BCE0FCA3E0FD7B017AF819
:1015200079C090F922E4F0A304F0227BFF90F8B890
:10153000E0FFA3E090F837CFF0A3EFF090F8BAE027
:10154000FFA3E090F839CFF0A3EFF090F8BCE0FFF4
:10155000A3E090F83BCFF0A3EFF012401490F8B95D
:10156000E04401FF90F8BBE0FD7B017AF879C09080
:10157000F929E4F0A304F022E4F0A37412F07BFF55
:101580007A1D792290F837F0124014227BFF7A1DE1
:10159000794C1240142212401490F8D6E004F02244
:1036BB0090F924EF12012490F924E0FE90F8D23017
:1036CB00E01AE0FFEE147AF9792590F90412010360
:1036DB00123769C0061200B7E4A3801EE0FF90F911
:1036EB0024E0FD7B017AF9792590F904E4F0A3122B
:1036FB003769C0061200B7A37402F090F8D2E0FF4E
:10370B001228BFD0E04F90F8D3F090F8D3E06026AA
:10371B0090F8D5E0FEA3E0FF1244BB1201804003FA
:10372B001201A990F8D8E004F0700690F8D7E004E5
:10373B00F012018E408190F8D3E0FF601B7BFF7A83
:10374B001E79CB1200AE90F92412015A90F925E0A4
:10375B00FFE412016A12401490F8D3E0FF2204F048
:0D376B00A3F01228BF90F8D3EFF0E0FE228B
:1035F70090F91CEFF0A3EC12012490F91CE0FE9067
:10360700F8D230E017E0FFEE1412369DC00690F9AD
:103617001CE090F91F1200BEE4A38019E0FF90F9A7
:103627001CE012369DC00690F91CE0FD90F91F12B0
:1036370000BFA37402F090F8D2E0FF1228BFD0E0D9
:103647004F90F8D3F090F8D3E0602690F8D5E0FEDD
:10365700A3E0FF1244BB12018040031201A990F8B6
:10366700D8E004F0700690F8D7E004F012018E401D
:103677008990F8D3E0FF60187BFF7A1E79CB1200A0
:10368700AE90F91C12015A90F91D120165124014EF
:1036970090F8D3E0FF22FD7B017AF9791D90F904B8
:1036A700E4F0A37402F0A314F01228BF90F8D3EF4C
:0436B700F0E0FE221F
:03000000023B20A0
:0C3B2000787FE4F6D8FD758153023B6706
:10028000E709F608DFFA8046E709F208DFFA803E60
:1002900088828C83E709F0A3DFFA8032E309F6084D
:1002A000DFFA8078E309F208DFFA807088828C83B5
:1002B000E309F0A3DFFA806489828A83E0A3F60869
:1002C000DFFA805889828A83E0A3F208DFFA804C43
:1002D00080D280FA80C680D4806980F2803380101A
:1002E00080A680EA809A80A880DA80E280CA803383
:1002F00089828A83ECFAE493A3C8C582C8CCC583FB
:10030000CCF0A3C8C582C8CCC583CCDFE9DEE780CA
:100310000D89828A83E493A3F608DFF9ECFAA9F049
:10032000EDFB2289828A83ECFAE0A3C8C582C8CC9F
:10033000C583CCF0A3C8C582C8CCC583CCDFEADEB8
:10034000E880DB89828A83E493A3F208DFF980CC1A
:1003500088F0EF60010E4E60C388F0ED2402B40413
:100360000050B9F582EB2402B4040050AF232345BA
:0603700082239002D0730D
:10037600BB010CE58229F582E5833AF583E022503C
:1003860006E92582F8E622BBFE06E92582F8E22286
:0D039600E58229F582E5833AF583E49322A0
:1003A300F8BB010DE58229F582E5833AF583E8F090
:1003B300225006E92582C8F622BBFE05E92582C83C
:0203C300F22224
:1003C500BC000BBE0029EF8DF084FFADF022E4CC1C
:1003D500F875F008EF2FFFEE33FEEC33FCEE9DECE5
:1003E500984005FCEE9DFE0FD5F0E9E4CEFD22ED2B
:1003F500F8F5F0EE8420D21CFEADF075F008EF2F75
:10040500FFED33FD4007985006D5F0F222C398FD65
:050415000FD5F0EA2202
:10041A00E88FF0A4CC8BF0A42CFCE98EF0A42CFC81
:10042A008AF0EDA42CFCEA8EF0A4CDA8F08BF0A4FF
:10043A002DCC3825F0FDE98FF0A42CCD35F0FCEB5E
:10044A008EF0A4FEA9F0EB8FF0A4CFC5F02ECD3923
:0F045A00FEE43CFCEAA42DCE35F0FDE43CFC2290
:1004690075F008758200EF2FFFEE33FECD33CDCC4A
:1004790033CCC58233C5829BED9AEC99E5829840CD
:100489000CF582EE9BFEED9AFDEC99FC0FD5F0D6AA
:10049900E4CEFBE4CDFAE4CCF9A88222B800C1B9D4
:1004A9000059BA002DEC8BF084CFCECDFCE5F0CB12
:1004B900F97818EF2FFFEE33FEED33FDEC33FCEB4B
:1004C90033FB10D703994004EB99FB0FD8E5E4F906
:1004D900FA227818EF2FFFEE33FEED33FDEC33FCF3
:1004E900C933C910D7059BE99A4007EC9BFCE99AE7
:1004F900F90FD8E0E4C9FAE4CCFB2275F010EF2F2C
:10050900FFEE33FEED33FDCC33CCC833C810D7072B
:100519009BEC9AE899400AED9BFDEC9AFCE899F866
:0E0529000FD5F0DAE4CDFBE4CCFAE4C8F922F9
:1040F500C2D5E830E70FB2D5E4C39BFBE49AFAE4F6
:1041050099F9E498F8EC30E717B2D512412B12046F
:10411500A5E4C39BFBE49AFAE499F9E498F88003D3
:104125001204A530D50DE4C39FFFE49EFEE49DFD7A
:04413500E49CFC22E8
:10053700E86010ECA2E713FCED13FDEE13FEEF13DA
:04054700FFD8F022C7
:0C054B00E6FC08E6FD08E6FE08E6FF22DC
:0D055700E6FB08E6F908E6FA08E6CBF82214
:0C056400ECF608EDF608EEF608EFF622C3
:10057000D083D082F8E4937012740193700DA3A31A
:1005800093F8740193F5828883E47374029368602E
:06059000EFA3A3A380DF2E
:060596008A838982E473F0
:10059C00E5132582F582E5123583F583B5120485C2
:1005AC0082132210AF06858213F51222858213F571
:0405BC0012D2AF2286
:0D05C000E5132582F582E5123583F58322CF
:10190500E508300C0104F823282465F582E434F851
:10191500F5832290F862300C0390F865E475F001C8
:101925001209C302094860EAC50C7002150B14C5FB
:101935000C200C04FF02451B90F86274FFF5F002C1
:1019450009DAFF02447BE5096006D509037F002219
:10195500200C0F124467EF6008050CE50C700205BA
:101965000B2290F8621209BA120948FF60E890F854
:1019750062E475F0011209C380DC121955EFC0E06D
:10198500121947D0E040F3809DD20C8002C20C9022
:10199500F8621209F1E4F50AF508F50BF50C75097D
:1019A50000C20BC209C20AC20D121918FF7005AF99
:1019B5000A7E0022B42530121918FF24D0B40A007B
:1019C500500C75F00AC509A42509F50980E924CF4D
:1019D500B41A00EF5002C2E5021BF3D20A80D8D236
:1019E5000980D4D20D80D0EF121947500812197F03
:1019F500EF600E80A9EFC0E0121955D0E06F609E30
:101A0500EF607412192B80A7121955EF6069E5096B
:101A1500700705098003121955EF6014200D0E1289
:101A25001905E475F0011209C3EF120961D509E63C
:101A3500200D040508050A80BA12194BEFC0E01203
:101A45001947D0E0500412192BE4FF200D0E12198E
:101A550005E475F0011209C3EF120961EF70DA2090
:101A65000D040508050A808BE509600205091219B0
:101A75007F12194BEF70C6300C04E412192BE50ADE
:101A850060030219B47EFF7FFF22200D1174FFFC55
:101A9500FDFEFF1219051209BA1209A0050802195F
:101AA500A3D0E080D27900800A7910800679088079
:101AB50002790AD20EE50960020509E9C0E01219AA
:101AC5007FEF60DD121955BF2D04D20B8003BF2BAC
:101AD5000912197FEF60CA12194BD0E0B40A0280CF
:101AE50033B40802802EBF302770027408C20EC0BE
:101AF500E012194BD0E0BF78028003BF58160509E4
:101B0500D509028007D50904D20E800B74108019FF
:101B15007002740ABF000AEFF8E4FCFDFEFF021B29
:101B2500A6C0E0EF12192BD0E0F9E4FCFDFEFFE9B9
:101B3500C0E0ECC0E0EDC0E0EEC0E0EFC0E012199F
:101B45004BEFF8D0E0FFD0E0FED0E0FDD0E0FCD0D8
:101B5500F0E8604DB461004007B47B005002C2E577
:101B650024D0503DFA24F6500724F95034240AFABB
:101B7500EAB5F000502BCFA9F0A42FFF92D5E9C507
:101B8500F0CEA4A2D53EFE92D5E9C5F0CDA4A2D54E
:101B95003DFD92D5E9C5F0CCA4A2D53CFCC20E8092
:061BA5008EE8C0E0200DF7
:101BAB002A200E08050A300B03120992121905128E
:101BBB0009BA050820090B200A0DEE8FF0120973E4
:101BCB0080091209A08004EF120961D0E012192BD1
:101BDB000219A3200D101219051209BA0508E50BFD
:101BEB00850CF012097380E81205701A6D531AAE4A
:101BFB005819E44C19E04219BC481AB24F1AB644B2
:101C0B001A0D431AAA491AB6551A8F461A8F451A36
:0C1C1B008F4719E82A1BDE4E000019EC70
:1005CD00E3F5F009E208B5F06D606B80F3E3F5F04B
:1005DD0009E608B5F060605E80F387F009E608B5BE
:1005ED00F054605280F487F009E208B5F048604697
:1005FD0080F488828C8387F009E0A3B5F0386036EB
:10060D0080F488828C8387F009E493A3B5F027608A
:10061D002580F388828C83E3F5F009E0A3B5F0160D
:10062D00601480F388828C83E3F5F009E493A3B51D
:10063D00F004600280F20206F8808580E7808E80EB
:10064D00D2803C8015806C807E809B80B5808B80B5
:10065D00A1804F8070803A02070E89828A83ECFA5E
:10066D00E493F5F0A3C8C582C8CCC583CCE493A3AD
:10067D00C8C582C8CCC583CCB5F070606E80E189E9
:10068D00828A83E493F5F0A3E208B5F05E605C80A6
:10069D00F289828A83E0F5F0A3E608B5F04D604B50
:1006AD0080F389828A83E0F5F0A3E208B5F03C601F
:1006BD003A80F389828A83E493F5F0A3E608B5F0D6
:1006CD002A602880F2805D89828A83ECFAE493F5B2
:1006DD00F0A3C8C582C8CCC583CCE0A3C8C582C869
:1006ED00CCC583CCB5F004600280E27F00F845F004
:1006FD00600EE863F0806480D395F01F40027F01A7
:10070D002289828A83ECFAE0F5F0A3C8C582C8CCB1
:10071D00C583CCE0A3C8C582C8CCC583CCB5F0CB0E
:10072D0060C980E389828A83ECFAE0F5F0A3C8C53D
:10073D0082C8CCC583CCE493A3C8C582C8CCC5837D
:10074D00CCB5F0A760A580E288F0ED2402B40400DA
:10075D005099F582EB2402B40400508F2323458277
:05076D00239006467315
:10000E00E4FFFE120948600C0FEF70010E09E97053
:05001E00F20A80EF2250
:10077200E3F5F009E208B5F06BDFF58067E3F5F029
:1007820009E608B5F05EDFF5805A87F009E608B59C
:10079200F052DFF6804E87F009E208B5F046DFF648
:1007A200804288828C8387F009E0A3B5F036DFF6B9
:1007B200803288828C8387F009E493A3B5F025DF29
:1007C200F5802188828C83E3F5F009E0A3B5F0146B
:1007D200DFF5801088828C83E3F5F009E493A3B5FA
:1007E200F002DFF40208A1808780E9809080D48043
:1007F2003E8015806E807E809D80B7808D80A38034
:10080200518074803C0208AD89828A83ECFAE493B9
:10081200F5F0A3C8C582C8CCC583CCE493A3C8C5F0
:1008220082C8CCC583CCB5F076DFE3DEE180708987
:10083200828A83E493F5F0A3E208B5F062DFF480E4
:100842005E89828A83E0F5F0A3E608B5F051DFF510
:10085200804D89828A83E0F5F0A3E208B5F040DF9B
:10086200F5803C89828A83E493F5F0A3E608B5F02B
:100872002EDFF4802A8002805789828A83ECFAE490
:1008820093F5F0A3C8C582C8CCC583CCE0A3C8C584
:1008920082C8CCC583CCB5F006DFE4DEE280007FFF
:1008A200FFB5F0020F2240027F012289828A83EC87
:1008B200FAE0F5F0A3C8C582C8CCC583CCE0A3C8D2
:1008C200C582C8CCC583CCB5F0D5DFE5DEE380CFE9
:1008D20089828A83ECFAE0F5F0A3C8C582C8CCC548
:1008E20083CCE493A3C8C582C8CCC583CCB5F0AF92
:1008F200DFE4DEE280A988F0EF60010E4E60ABED2E
:100902002402B404005098F582EB2402B40400508F
:0A0912008E23234582239007E9732A
:10091C00EF4E6012EF60010EEDBB010B89828A83F2
:10092C00F0A3DFFCDEFA2289F05007F709DFFCA9FF
:0C093C00F022BBFEFCF309DFFCA9F02256
:1040AB0090F92BE0FFA3E0FEA3E0CF90F893F0A3F1
:1040BB00EEF0A3EFF090F92EE0CBF0A3E0CAF0A363
:1040CB00E0C9F07F2290F896AD82AC831209488D3F
:1040DB00828C83F0A309E970010ADFEC90F92EE0E2
:0A40EB00FBA3E0FAA3E0F9021605BA
:103B2C00020A12E493A3F8E493A34003F68001F293
:103B3C0008DFF48029E493A3F85407240CC8C3339A
:103B4C00C4540F4420C8834004F456800146F6DF69
:103B5C00E4800B0102040810204080903D39E47E83
:103B6C00019360BCA3FF543F30E509541FFEE4935E
:103B7C00A360010ECF54C025E060A840B8E493A325
:103B8C00FAE493A3F8E493A3C8C582C8CAC583CA50
:103B9C00F0A3C8C582C8CAC583CADFE9DEE780BE08
:013DB400000E
:10094800BB010689828A83E0225002E722BBFE02AD
:09095800E32289828A83E49322E0
:10096100BB010689828A83F0225002F722BBFE0175
:02097100F3226F
:10097300BB010A89828A83F0E5F0A3F0225006F7CF
:0F09830009A7F01922BBFE06F3E5F009F31922CC
:0E099200C3E49FFFE49EFEE49DFDE49CFC2276
:1009A000BB010789828A830209FA5005E9F802052A
:0A09B00064BBFE05E9F8020A062206
:0909BA00E0FBA3E0FAA3E0F9223E
:1009C300F8E0FBA3A3E0F925F0F0E58215827002BD
:0709D3001583E0FA38F02261
:1009DA00F8E0FBA3A3E025F0F9F0E58215827002A6
:0709EA001583E038FAF0224A
:0909F100EBF0A3EAF0A3E9F02207
:1015A000E50D2493F582E434F8F583E0050D2290EF
:1015B000F89030070390F893E475F0011209C30224
:1015C00009482000E97F2ED2008018EF540F2490A4
:1015D000D43440D4FF30040BEF24BFB41A005003BE
:1015E0002461FFE50E6002150E0511E5117002057C
:1015F0001030070E90F890E475F0011209C3EF0265
:1016000009610242F27403D2078003E4C207F50DB8
:1016100090F8901209F1E4F50EF510F511E50E6061
:10162000077F201215E380F5750FFFC201C200C2CB
:1016300002C203C205C206C2081215AFFF700D3008
:1016400007057F001215F4AF11AE1022B4255FC25A
:10165000D5C2041215AFFF24D0B40A00501A75F099
:101660000A780E30D50508B6FF0106C6A426F62076
:10167000D5047002D20380D924CFB41A00EF5004ED
:10168000C2E5D2040217F5D20180C6D20080C0D2D2
:101690000280BCD2D580BAD20580B47F201215E377
:1016A0002002077401B50E0040F11215A0FF1215BB
:1016B000E302161DD208D20680951215A0FB121562
:1016C000A0FA1215A0F94A4B700679C67A187BFF6A
:1016D00020022EE50E602A7E008E827583001203A2
:1016E0007660060EEE650F70F0C2D5EBC0E0EAC082
:1016F000E0E9C0E0EE12183CD0E0F9D0E0FAD0E02A
:10170000FB120948FF60AAEBC0E0EAC0E0E9C0E0D4
:101710001215E3D0E02401F9D0E03400FAD0E0FB68
:10172000E50F0460DCD50FD980877BFF7A18793804
:10173000D202809C791080027908C206C208800813
:10174000D2D5790A8004790AC2D5E50F047002F572
:101750000FE4FAFDFEFF1215A0FC7B082001131216
:1017600015A0FD7B1030000A1215A0FE1215A0FF77
:101770007B20EC3382D592D55013C3E43000069F12
:10178000FFE49EFEE42001039DFDE49CFCE4CBF815
:10179000C201EC700CCFCECDCCE824F8F870F38009
:1017A00017C3EF33FFEE33FEED33FDEC33FCEB33C9
:1017B000FB994002FB0FD8E9EB300105F8D0E0C4FB
:1017C00048B201C0E00AEC4D4E4F78207B0070C259
:1017D000EAB50F0040BCC0E012183ED0F0D0E020C7
:1017E0000104C4C0E0C4B201C0F01215CCD0F0D5E1
:1017F000F0EB02161D12057016BA53173458168BEB
:101800004C16874217384F17404417404916A043DB
:08181000174655172A46172A56
:1018180045172A4718E650168F2D16932E16B62B05
:1018280016972316B42018CF2A164F48000016AE74
:101838003F3F3F00790AA2D5200314300509B910AB
:10184800020404B9080104A2D520060250010420AC
:1018580002689202B50E005034C0E07F20300319B0
:101868007F30A20272067205500F121895C202C28A
:1018780006C205C2087F30800F300503E9C0E012B8
:1018880015E3300503D0E0F9D0E0B50ECC300517EC
:101898007F30B9100C1215E37F583004077F788029
:1018A80003B908031215E33002057F2D0215E37F03
:1018B800202008F87F2B2006F322920280CF286E82
:1018C800756C6C2900D2011215A03001F8C201789C
:1018D8000E30D50108F602164F2D504349581215FF
:1018E800A02403B405004001E49018E1931215D434
:0D18F800743A1215D4D203750E0402173491
:1044670010140B124501BF0D027F0A0242F290F9A8
:044477005FE0FF22E1
:08451B0090F95FEFF0D21422C9
:10447B00EFC394094005EF940E4004EFB42003D32F
:04448B008001C322C7
:0C09FA00ECF0A3EDF0A3EEF0A3EFF02270
:0C0A0600ECF208EDF208EEF208EFF2222C
:1042F200EFB40A07740D1242FD740A309811A8999E
:10430200B8130CC2983098FDA899C298B811F6302B
:0743120099FDC299F5992203
:0A4501003098FDAF99C2987E0022A9
:00000001FF
